:1080000038450020D9A20000F1A20000F3A2000030
:10801000F5A20000F5A20000F5A20000000000009B
:10802000000000000000000000000000F5A20000B9
:10803000F5A2000000000000F5A20000A5910000DC
:10804000F5A20000F5A20000F5A20000F5A20000D4
:10805000F5A20000F5A20000B79D0000F5A2000007
:10806000F5A20000F5A20000F5A20000F5A20000B4
:10807000F5A20000F5A20000F5A2000011830000A7
:10808000F5A20000F5A20000F5A20000F5A2000094
:10809000F5A20000F5A20000F5A20000F5A2000084
:1080A000F5A20000F5A20000F5A20000F5A2000074
:1080B000F5A20000F5A20000F5A20000F5A2000064
:1080C000F5A20000F5A20000F5A20000F5A2000054
:1080D000F5A20000F5A20000F5A20000F5A2000044
:1080E000F5A20000F5A2000000000000F5A20000CB
:1080F000F5A20000F5A20000F5A20000F5A2000024
:10810000F5A20000F5A20000F7830000F5A2000030
:108110000000000000000000F5A20000F5A2000031
:10812000F5A20000F5A20000F5A20000F5A20000F3
:10813000F5A20000F5A20000F5A20000F5A20000E3
:10814000000000000000000000000000000000002F
:10815000F5A20000F5A20000F5A20000F5A20000C3
:10816000000000000000000000000000000000000F
:1081700000000000000000000000000000000000FF
:1081800000000000000000000000000000000000EF
:1081900000000000000000000000000000000000DF
:1081A00000000000000000000000000000000000CF
:1081B000F5A20000F5A20000F5A20000F5A2000063
:1081C000F5A20000F5A20000F5A20000F5A2000053
:1081D000F5A20000F5A20000F5A20000F5A2000043
:1081E000F5A20000F5A20000F5A2000000000000CA
:1081F00000000000F5A20000F5A20000F5A20000BA
:10820000F5A20000F5A20000000000000000000040
:10821000F5A20000F5A20000F5A20000F5A2000002
:10822000F5A20000F5A20000F5A20000F5A20000F2
:10823000F5A20000F5A20000F5A20000F5A20000E2
:10824000F5A20000F5A20000F5A20000F5A20000D2
:10825000F5A20000F5A20000F5A20000F5A20000C2
:10826000F5A20000F5A20000F5A2000070B52021E3
:10827000DFF8C00800F077FD0020DFF8BC180860C8
:108280002021DFF8B80800F06EFD0020DFF8B018FC
:10829000086000F0EEFA00F0A4FA00F073FB03238C
:1082A00006220121DFF89C0800F005FEDFF898683F
:1082B00040F21B303060DFF894484FF44770206084
:1082C00000F0AEFE050000F0ABFE401BB0F5FA7FFB
:1082D000F9D36420DFF8781809684143326891FBCC
:1082E000F2F1DFF870281160DFF86C18096800FB04
:1082F00001F0216890FBF1F0DFF8601808600520BC
:10830000DFF85C1808700120DFF85818086070BDAD
:1083100038B50220DFF850180860DFF8500802680E
:108320000168DFF84C381B689B0709D4DFF8443834
:108330001B689B0704D4DFF840381B68DB051BD49F
:10834000DFF80048216831F00201216000E0016897
:10835000DFF824180968C905F9D5DFF8E8570121C5
:10836000280000F013FE0121280000F015FE20680F
:1083700050F0020020603DE0DFF8004823680F2045
:1083800000FB0322102092FBF0F32360DFF8C027EC
:10839000DFF8C00700681B1ADFF8AC07006843432A
:1083A000642093FBF0F01060DFF8D4371C680F20D6
:1083B00000FB0411102091FBF0F11960DFF89837F1
:1083C000DFF898070068091ADFF880070068414362
:1083D000642091FBF0F01860DFF8A807006800281F
:1083E00004D41068DFF8A017086003E01868DFF80D
:1083F0009817086031BDDFF89407002101605FF431
:108400008021DFF88C271160FF22DFF888371A609F
:108410000160DFF88407016851F0020101607047D4
:10842000DFF874070068002801D1002000E0012077
:1084300070470120DFF8641708607047DFF82407F1
:108440000068002804D10020DFF8F416086003E07B
:108450002020DFF8EC16086070470020DFF8E016F7
:10846000086070472DE9F0410C00DFF8F816096844
:10847000002904D005002800C0B2072806DBDFF879
:108480001807016851F004010160A8E1DFF8D06627
:1084900028003178C0B2884200F0ED802800C0B2D8
:1084A000062803D13078022800F0E5802800C0B209
:1084B000022803D13078062800F0DD802800C0B201
:1084C000022803D02800C0B2062818D1DFF8D076E1
:1084D00000220321380000F0D6FE00220C213800D3
:1084E00000F0D1FE00F0C5F901220321380000F0B0
:1084F000CAFE01220C21380000F0C5FEA3E02800CE
:10850000C0B2052804D10020DFF82C1608609AE0DC
:108510002800C0B2002812D12020DFF81C16086005
:10852000DFF87C7600220321380000F0ACFE002248
:108530000C21380000F0A7FE00F09BF983E0280032
:10854000C0B201281CD1DFF8587600220321380080
:1085500000F099FE00220C21380000F094FE00F09B
:1085600088F901220221380000F08DFE0122082145
:10857000380000F088FE2020DFF8BC15086062E0BB
:108580002800C0B2042835D1DFF814760022032178
:10859000380000F078FE00220C21380000F073FE55
:1085A000DFF80076C021380000F0DDFB3021380014
:1085B00000F0D9FB00224021380000F0B7FB8022F8
:1085C0008021380000F0B2FB00221021380000F0BA
:1085D000ADFB20222021380000F0A8FB2020DFF88E
:1085E00058150860002300220121DFF8580500F02B
:1085F00062FC28E02800C0B203281ED100F039F93F
:10860000DFF89C754FF4FA624021380000F017FE45
:108610004FF4FA628221380000F011FE0321380085
:1086200000F02CFE01220321380000F02CFE012274
:108630000C21380000F027FE05E0DFF85C0501683A
:1086400051F0040101602800C0B2042803D02800C2
:10865000C0B2052807D1002300220121DFF8E4047D
:1086600000F029FC36E0002306220121DFF8D404C3
:1086700000F021FC2EE02800C0B2052821D1002006
:10868000DFF8B4140860DFF8187500220321380001
:1086900000F0F9FD00220C21380000F0F4FD00F09C
:1086A000E8F801220221380000F0EDFD0122082146
:1086B000380000F0E8FD0121DFF8880400F072FCCA
:1086C00008E02800C0B2042804D10121DFF87404B6
:1086D00000F068FC20002900C9B2022963D1DFF84C
:1086E000A484C8F80000D8F8004014F5FA64DFF854
:1086F000B07422004021380000F0A1FD2200822148
:10870000380000F09CFDD8F8000000280CD44FF48D
:1087100080724021380000F0E0FD4FF400724021EB
:10872000380000F0D4FD0BE04FF400724021380017
:1087300000F0D3FD4FF480724021380000F0C7FDF7
:108740000321380000F09AFDDFF83C040168642939
:1087500015DADFF854140968012910D100F060FC23
:10876000DFF848140968401A40F6B931884215D339
:10877000DFF82404016851F0010101600EE0006897
:1087800040F2F511884204DB0020DFF81C14086079
:1087900004E000F045FCDFF8141408600020DFF866
:1087A000101408601AE02900C9B2062902D100F0AD
:1087B0004FF913E000F034FCDFF8F01308600120FB
:1087C000DFF8E4130860DFF8D4030168012905D15C
:1087D0000021DFF8C4231160002101603570BDE87D
:1087E000F08110B5DFF8CC0300F0A0FDD14C0421DE
:1087F000200000F09FFA0221200000F09BFAD14CEB
:108800000021200000F003FC0720DFF8AC13086013
:108810001F2000F05DFF0121200000F035FB012149
:10882000200000F040FB002306220121200000F080
:1088300042FB012300220121200000F066FB62239D
:1088400001220121200000F060FB0121200000F046
:1088500025FB0121200000F01AFB1F2000F00CFF77
:108860000121200000F09EFB00211F2000F0F3FEFC
:1088700010BD38B5D14800F059FDD14800F09DFA3F
:10888000D04800F09AFAD04800F097FACF4800F0AC
:1088900094FAC44C4021200000F073FA802120009B
:1088A00000F06FFA1021200000F06BFA2021200068
:1088B00000F067FABA4CC64D2A004021200000F0B3
:1088C0009BFC2A008021200000F096FCE020C1499A
:1088D0000860B020C0490860AA20C04908604FF471
:1088E0007A624021200000F09DFC4FF47A628021E2
:1088F000200000F097FC4021200000F09DFC80212A
:10890000200000F099FC0321200000F0B9FC5FF486
:108910007020B349086000220F21200000F0C5FC40
:1089200001220F21200000F0C9FC00220F212000AD
:1089300000F0A9FC00220F21200000F0ADFC4FF454
:10894000FA624021200000F07AFC4FF4FA628221A2
:10895000200000F074FC0E230E224021200000F0C5
:1089600080FC0E230E228021200000F07AFC0321DF
:10897000200000F083FC4FF400724021200000F042
:10898000A6FC31BD70B56B4C0421200000F0D2F97B
:108990000221200000F0CEF9924C200000F0C6FC2D
:1089A000200000F0DDFC422000F092FE8E4C0221FF
:1089B000200000F069FA0221200000F074FA002182
:1089C000200000F024FB07208849086002212000D5
:1089D00000F00CFB40F6AC5540F6D86633002A0098
:1089E0000021200000F0FAFA33002A0001212000C3
:1089F00000F0F4FA41F61D552A000021200000F095
:108A0000E7FA2A000121200000F0E2FA20212000EC
:108A100000F0D6FA03230F220221200000F04BFAC7
:108A2000734B00220221200000F06FFA714B0122EB
:108A30000221200000F069FA0221200000F02EFA45
:108A4000422000F019FE0221200000F0D4FA70BD8F
:108A500070B50500564E280000F0F6FE30604A4C16
:108A600030682168884226DA6348006821688842B5
:108A700021D020683168411A4FF47A704143206850
:108A800091FBF0F13F4A106841434FF47A7091FB3B
:108A9000F0F01168081A1060106840F26D71884299
:108AA00003DB40F26C70106040E054481168814272
:108AB0003CDA10603AE020683168B1F5C87188424C
:108AC00008DB20683168884230DA4B48006821684A
:108AD00088422BD130682168411A4FF47A704143A3
:108AE000206891FBF0F1274E306841434FF47A70D3
:108AF00091FBF0F000F0A8FE0A2800DA0A20002D11
:108B000003D431684018306002E03168081A3060E0
:108B1000306840F26D71884203DB40F26C70306067
:108B200004E036483168814200DA3060206832491A
:108B3000086070BD0040024080400240007000406C
:108B400080700040008003401005002014050020C4
:108B5000FC04002008050020000500200C05002072
:108B600034050020F00400200C800340688003409E
:108B700010800340188003406C80034024050020CF
:108B80002805002018050020040500200890034057
:108B90000C90034034900340EC040020F8040020C3
:108BA0000080024000500040F40400202005002016
:108BB0001C050020003800F0C48F0340004000F086
:108BC00004180100041C0100041001000414010039
:108BD000BAAA050060800240A080024028800240BE
:108BE0001C800240013800F000900340C49F034005
:108BF00001000800220009002C05002094F8FFFF66
:108C000030B5CB4300F58064D50725684CBF0D43D4
:108C10001D40256000F58460920747BF026811433C
:108C200001681940016030BDF0B5002400F6C4753C
:108C30000126A640314211D066002F684FF0030C88
:108C40000CFA06FC27EA0C072F60C2F34117D5F88F
:108C500000C007FA06F646EA0C062E60641C082CD3
:108C6000E6DBCC4300F5A065D6072E684CBF0E436B
:108C700026402E6000F2045596072E684CBF0E4326
:108C800026402E6000F5A16556072E684CBF0E43A6
:108C900026402E6000F5A36516072E684CBF0E43D4
:108CA00026402E6000F23C55D2062A684CBF0A438B
:108CB00022402A60DD0700F20C5215684CBF0D43BC
:108CC0002540156000F5A2629D0715684CBF0D4355
:108CD0002540156000F214525D0715684CBF0D4326
:108CE0002540156000F21C521D0715684CBF0D434E
:108CF0002540156000F244529D0515684CBF0D4398
:108D00002540156000F5A86213F4407F156814BF74
:108D10000D432540156000F5A560002B07BF0268D4
:108D200041EA020401680C400460F0BD00EB8100E0
:108D30000260704738B5FFE704460D460022FFF792
:108D40005FFF2946204601B0BDE8304000230122E4
:108D50006AE738B500F02DF82946204601B0BDE895
:108D600030400823F3E738B504460D460823FFE7F3
:108D70000122FFF759FF29462046BDE8384001226D
:108D80003EE738B500F007F82946204601B0BDE8B7
:108D900030400823DBE704460D46022230E738B5B1
:108DA000FFF7F9FF2946204601B0BDE8304008230F
:108DB000CDE704460D46002222E710B50D4B0FF219
:108DC00038021C68C0F30741CC40E40746BF02EB01
:108DD000C101496852F8311001F22C51020A0B68A6
:108DE0000F24944000F00F00A34390401843086004
:108DF00010BD00006CE00F400040004000800540C6
:108E000000500040009005400060004000A0054078
:108E10000070004000B005400040024000C0054026
:108E20000050024000D005400060024000E00540D4
:108E30000070024000F0054000D0034000000640F2
:108E400000100640001006400020064000200640AA
:108E5000003006400030064000400640004006401A
:108E6000005006400050064000600640006006408A
:108E700000700640007006400080064000800640FA
:108E8000009006400090064050F8082F0CE00122A8
:108E900002FA01F100F10C021160B3E00268012353
:108EA00003FA01F1B0E00268012303FA01F122EABA
:108EB000010101607047F0B500F1140689000F252B
:108EC0008D403468ED4302F00F0705EA040C07FA01
:108ED00001F444EA0C04346003F0030300F12004BD
:108EE00003FA01F126683540BF1F2943032F216093
:108EF0000AD8FF0050F81C1F3023BB4002F030029C
:108F00009943BA400A430260F0BD70B5490140314F
:108F1000081892000F2191400468C94303F00F051F
:108F20000C4095402C430460C3F3032600F1180461
:108F3000964025680D4035432560041DC3F3031694
:108F400000F01EF800F11C04C3F3035600F018F8FB
:108F50000124944013F4702F00F110050BD050F849
:108F6000146FC3F30243314003FA02F20A43026072
:108F70002868044302E0286820EA04042C6070BDDD
:108F800025680D409640354325607047012202FA5E
:108F900001F140F8101F7047012202FA01F140F878
:108FA000181F704710B50B0C012401F00F0150F889
:108FB000282F04FA01F141EA03411143016010BD79
:108FC000002200E0521C4908FCD140F8302F7047C5
:108FD00000EB810000F560600260704700EB8100EB
:108FE00000F5646042EA03420260704750F8082FBF
:108FF0004FF4803359E750F8082F4FF4803303FAC9
:1090000001F101E050F8082F11430160704750F85A
:10901000382F920841EA820101607047872070472B
:1090200063480068704738B500F00EFB4FF400400D
:109030006049086000F02AFC5F4800F09FF90120B9
:1090400000F098F95D4C200000F070F95C4800F0E9
:109050006DF95C4D280000F069F95B4800F066F995
:109060005A4800F063F95A4800F060F9594800F096
:109070005DF900F043FC200000F074FA280000F0D5
:1090800071FA554800F0D4FC00F0C6FC00210F2016
:1090900000F0E1FA0F2000F0EFFA00F0C3FC00F05E
:1090A000CFFA4E4800F042F900F0CAFC4C4800F0FC
:1090B000DCFC4C4C10212000FFF755FE08236622F3
:1090C00010212000FFF7B0FD002047490860474C01
:1090D00040221021200000F02EFC206845280BD1F2
:1090E0006068312808D1A068342805D1E0683028AC
:1090F00002D12069302802D0102000F04AFD04225D
:109100000421684600F017FC9DF80000342803D1C4
:109110009DF8010032280CD034208DF80000322058
:109120008DF8010004220421684600F019FC002893
:10913000F8D15FF0704000F0F9F85FF0804000F087
:1091400049FD012803D15FF0804000F03BFD284934
:109150005FF0804000F045FD5FF0804000F027FDAB
:109160005FF0804000F045FD5FF0804000F01EFDA4
:109170005FF0804000F021FD31BD80B55FF08040A0
:1091800000F028FD012803D15FF0804000F01AFDB7
:1091900018495FF0804000F024FD5FF0804000F04F
:1091A0000CFD01BD02480168491C016070470000C8
:1091B0003005002008ED00E0800300C1000800F049
:1091C000010800F0020800F0030800F0040800F0B5
:1091D000050800F0005800F080380100000C00F095
:1091E0000000002000500240405002408004002057
:1091F00000B4C40400350C00401801686FF352013C
:109200001143016000F124012030920704D5B022FF
:1092100002604FF4306003E08C22026040F60C00E4
:1092200008607047401800F11001006883074CBFC8
:109230005208521E0A607047081801681AE010B5FB
:109240008B0900EB831003689C0700F1100348BFF3
:1092500052081B689A1AC9074CBF1C3018300260AC
:1092600010BD401800F12C010A6000F130010B60C4
:1092700050F8281F41F001010160704701607047FC
:1092800040F8041F70470830012A02680CBF1143E0
:1092900022EA0101016070470C30012A02680CBF0C
:1092A000114322EA0101016070472430012A02685B
:1092B0000CBF114322EA0101016070471030012AFE
:1092C00002680CBF114322EA0101016070470818CF
:1092D00050F8041F0A4302607047081850F8041F32
:1092E00021EA02020260704718B58100DFF88C2283
:1092F000C0F3072301F47F71D31841EA431343F00D
:10930000844301241C600023009302E0009C641C41
:109310000094009B102BF9D3C0F30720121841EAE8
:10932000421141F084410020086011BDC0F30722C2
:10933000DFF84C1280008A1800F47F7040EA421077
:1093400040F0844001210160704780008A1800F4D9
:109350007F7040EA421040F0844000210160704775
:10936000C0F30722DFF81C12EFE700000138FDD13F
:1093700070477047DFF814120860704770B5DFF867
:1093800008221369146A014623F4800301F00105E1
:1093900043F4006303F0010085F0010544F4006428
:1093A0001361284214620ED061F0010003404FF4B3
:1093B0008070906013614FF400201568EE054AD468
:1093C000401EFAD170BD080960F30A13DFF8CC0122
:1093D00013610440DFF8C80108400443C80000F0EE
:1093E000400004431462480B60F34D3360F34D3486
:1093F00040209060002C47BF146213611361146217
:10940000DFF8A0010340DFF8A00108400343C80DC6
:1094100060F3DC54480008D5DFF8900124F48004A0
:10942000084043F48003044301E024F0804408052D
:109430000BD44FF400405E490D68EE0701D4401E86
:10944000FAD123F4006324F4006413611462102041
:10945000BDE870408AE70028B5D170BDF0B5554928
:109460000A6D0B6E002B4CBF03F0700002F0300051
:1094700040B1102847D0202847D0302847D0702846
:1094800048D04AE00FF24C10C2F3841450F8245034
:10949000494C04EA0306B6F1004F4FF0FF3003D009
:1094A000002B41D416053FD43A4E376876680968D8
:1094B000C6F3042C06F01F060CF1010C761C16FBFB
:1094C0000CF67600B5FBF6F5C7F30906C7F3892756
:1094D0006F4301F47041BF0AB1F5005F06FB0575EB
:1094E00042F480020DD0B1F5405F18D0B1F5804F45
:1094F00017D0B1F5E04F16D0B1F5104F08BF2F4887
:1095000012E02F4810E0224DC2E72E4DC0E747F28F
:109510003055BDE74FF40045BAE70020F0BD2A48BA
:1095200002E02A4800E01C48510217D5002B10D554
:1095300059000BD51C40B4F1004F03D0002B05D4CB
:10954000110503D46D00C3F3865104E0C3F3C55184
:1095500001E0C2F3C351491CB5FBF1F5A84288BF35
:109560002846F0BD1A4901230A6800F00F0003FAEB
:1095700000F000E00A6810430860704700E50F4003
:1095800000E60F4000E80F4050E00F407CE00F4045
:109590000024F40060E10F4040787D018FFFFF7FE1
:1095A00030000080FEFF3FF80100C007000040408F
:1095B00068E10F4010E00F4000080080002D3101ED
:1095C00000B4C40400093D0080F0FA02005A6202AF
:1095D0006CE00F4040420F0000201C0080841E0001
:1095E00000802500999E36000040380000093D00AB
:1095F00000803E0000004B00404B4C0000204E001D
:10960000808D5B0000C05D000080700000127A0059
:1096100000007D0080969800001BB7000080BB0012
:10962000C0E8CE00647ADA000024F4000000FA00FA
:1096300080A81201002D310100366E0140787D01B5
:1096400080B500F0E1FA02E080B500F0D9FA00B18F
:109650000120C0B202BD10B50FF2D402830852F847
:1096600023201368C00000F01800FF248440A343A7
:1096700081401943116010BD04282B4903D10868AB
:1096800040F480300BE0052804D10A6842F400322F
:109690000A607047062804D1086840F480200860FA
:1096A00070470F2805D12148016841F0020101608F
:1096B00070470CD90FF21413A0F1100110384009B3
:1096C00053F82000012201F01F018A400260704718
:1096D0000428154903D1086820F480300BE00528E0
:1096E00004D10A6822F400320A607047062804D1C7
:1096F000086820F48020086070470F2805D10B48C7
:10970000016821F00201016070470CD90FF2D0030B
:10971000A0F110011038400953F82000012201F097
:109720001F018A400260704724ED00E010E000E075
:109730000000000018ED00E01CED00E020ED00E06E
:1097400000E400E004E400E008E400E00CE400E0F1
:1097500010E400E014E400E018E400E01CE400E0A1
:1097600020E400E024E400E028E400E02CE400E051
:1097700030E400E034E400E038E400E03CE400E001
:1097800040E400E044E400E048E400E04CE400E0B1
:1097900050E400E054E400E058E400E05CE400E061
:1097A00060E400E064E400E068E400E06CE400E011
:1097B00070E400E074E400E078E400E07CE400E0C1
:1097C00080E400E084E400E088E400E000E100E000
:1097D00004E100E008E100E00CE100E010E100E05D
:1097E00080E100E084E100E088E100E08CE100E05D
:1097F00090E100E000210100C9B230390A2902D20B
:109800003038C0B208E00100C9B24139062902D29D
:109810003738C0B200E00020704710B402000120C9
:10982000002302E0D45C00195B1C8B42FAD3C043D6
:1098300000F0FF0010BC704710F00F000149085CF9
:10984000704700004CA30000002801D54042FFE70C
:10985000704730B4002513E050F8042BD30744BF01
:10986000A9F101039A18091F042942F8045BFAD2EE
:1098700013468C0744BF15809B1CC90748BF1D7049
:1098800050F8041B0029E7D130BC7047024801683A
:1098900041F040410160704734EF00E038B50446C4
:1098A00000F029F8544D0321296000F024F801202C
:1098B000E40900FA04F45148E443046000F01BF8A2
:1098C000002028600A20BDE83240FFF74FBD10B5E8
:1098D00000F011F8484C0321216000F00CF84749D2
:1098E0000020086000F007F8002020600A20BDE892
:1098F0001040FFF73BBD0A20FFF738BD10B502202E
:10990000FFF734FD3E4C2168C807FCD4606810F0B6
:109910000C0F0CD13B48FFF7E7FC0220FFF726FDB8
:109920002068C107FCD4606810F00C0F01D0022041
:1099300010BD002010BD10B5334B8C091C60C1F365
:109940008301920859600AD004E0596811B91C6873
:10995000641C1C60521E196940F8041BF5D110BD2F
:109960002DE9F84F81468A46274D6869C007FCD427
:10997000DFF89880264F274E4FEA9A102860940807
:10998000CAF38300686005D12AE0686810B92968C5
:10999000491C296030683840404505D130680104D1
:1099A00004BF5046FFF77AFFD9F800002861FFF79F
:1099B000A2FFD5F814B05FEACB70FAD45FEACB60AF
:1099C0000AD530680740474504D13068010408BF14
:1099D000FFF77DFF58460DE0641E09F10409D4D15C
:1099E00030680740474504D13068010408BFFFF7DD
:1099F0006EFF6869BDE8F28FFCD00F40C0E20A40FC
:109A000018F00A40005800F004F00A400000051069
:109A10000000FF7000E00F400748016841F00501B9
:109A2000016070470448016841F00201016070471D
:109A30000249401E0860704710E000E014E000E0BA
:109A40004349FFE7012008607047012100F01F0033
:109A500001FA00F03F4908607047012100F01F0043
:109A600001FA00F03C49086070473C4908607047C3
:109A700000F01F00012202FA00F0394ACB0748BF6C
:109A800010608B0748BF90614B0748BF1062090701
:109A900048BF90607047314A126800F03F0002EB07
:109AA0000012304893680340194391607047F0B545
:109AB0002A4C25682C4C00F03F0005EB0016B768D7
:109AC0002740840604D5042914BF062941F001016A
:109AD000DDF814C0ACF1010E41EA0E14274307F083
:109AE0004064B4F1406F04D0A40E0CFA04F4A21840
:109AF000521E326007F04042B2F1404F0FD00429AD
:109B000018BF062906D140F0200005EB001000F137
:109B10000C0304E0920F0CFA02F003445B1E736026
:109B2000B760F0BD11480068704700F0FF0110B544
:109B3000CB080F4A02EB8302890001F01C01136875
:109B40000F248C40000CA34388401843106010BDC4
:109B500004F00F4028F00F402CF00F4008F00F40A9
:109B60001CF00F40F73FFC0008C0FFFF04F50F405A
:109B700010F50F4080B50C4A1368010089B28B4381
:109B800013604FF6FF7180B2884201D1FEF751FC9D
:109B900001BD05490A6880B2104308607047024958
:109BA000096880B208407047D00400201BE050F8DC
:109BB000081F41F002010160704700F5406001217B
:109BC0000160704700F54060014901607047000086
:109BD00051E5CC1A00F540600068012818BF00204C
:109BE00070470160704750F8081F41F001010160A3
:109BF000704700F58360016841F48071016070472F
:109C0000EFF3108072B67047EFF3108062B67047C2
:109C100010B5DFF8EC03FFF789FBDFF8E803FFF787
:109C2000CCF8DFF8E403FFF7C8F83021DFF8DC03F5
:109C3000FFF7B5F8FFF712FCDFF8D44360235FF4B9
:109C4000E1320100200000F00FFA10220221200072
:109C500000F006FA1021200000F059FA200000F070
:109C600032FA0321200000F060FA1620FFF75DFFB2
:109C70001720FFF75AFFC0211620FFF7ECFC162033
:109C8000FFF7FAFC0F211620FFF7F2FEDFF884132E
:109C90001620FFF700FF0F211720FFF7E9FEDFF87E
:109CA00078131720FFF7F7FE4FF40070FFF771FFEE
:109CB0004FF48070FFF76DFF00F04AF9FFF7B0F93D
:109CC000DFF8581308600120DFF85413086010BD56
:109CD00038B5DFF84C03006800286BD0FFF7A0F917
:109CE000DFF838432168401A652807D34FF48070A5
:109CF000FFF74FFF00210520FEF7B4FB00F0B9F895
:109D0000012857D1C74D6878BB2803D1C648C74939
:109D10000860FBE7A878C0281FD1FFF781F9206011
:109D20004FF48070FFF726FFE978287970F0FF0084
:109D3000042907D1C043002804D04FF40070FFF776
:109D400019FF03E04FF40070FFF723FF00F044F821
:109D500000210520FEF786FB2CE0C1282AD12979B5
:109D6000687951EA0021A87951EA0041E87951EA7D
:109D70000061E878FEF776FB2D7AE80702D4FEF75B
:109D80006CFB01E0FEF75AFBFFF74AF920604FF445
:109D90008070FFF7EFFEA80703D5A348A34908602A
:109DA000FBE7680703D54FF6FF70FFF7E3FE0120DE
:109DB00000F02CF831BD10B5954C0121200000F0C9
:109DC000ABF90100200000F0ADF9FFF7ABFE400257
:109DD00001D500F0BDF810BD10B5954C05202070E0
:109DE00000206070C020A070FFF718F9E070E078E4
:109DF000C0432071342060713220A0718D4C00F07E
:109E0000C4F82060206800F0B4F810BD10B5884C8C
:109E10000821217000216170C221A170012802D1A6
:109E20000020E07001E0FF20E070FEF7F9FA012861
:109E300003D10220FFF7ADFE02E00220FFF79AFEF9
:109E40004FF6FF70FFF7ABFE20710100090A617148
:109E50000100090CA171000EE071002020720020A9
:109E60006072744C00F091F82060206800F081F876
:109E700010BD70B54FF480752C00002000E0401C30
:109E8000B0F5807F06DA6C490A5C032AF7D100221C
:109E90000A540400B4F5807F01D1002057E000206F
:109EA00004E0002050540C000020401CB0F5807FDE
:109EB0000DDA211A491E01F0FF015F4A535C032BA2
:109EC000EFD0535C022BF0D1002050540D00B5F5BB
:109ED000807F01D100203AE0641B04F0FF04641E7F
:109EE000072C01D2022032E0E00701D502202EE04B
:109EF0006408002C01D0802C01D3022027E000262A
:109F00000FE015EB4600401C00F0FF00411C01F083
:109F1000FF01494A515C105C00F092F841498855B4
:109F2000761CA642EDD33F4D2878E11E884201D031
:109F300002200CE0A11E681CFFF76FFC05EB04017A
:109F400011F8011C884201D0022000E0012070BD00
:109F500080B51620FFF781FD4FF480700090364BDE
:109F60002B4A01211620FFF7A2FD1620FFF76DFDF9
:109F700001BD80B50090264B304A01211720FFF724
:109F800096FD1720FFF761FD01BDF8B501262B4DA9
:109F900002202870002415E0385DC0B20009C0B26C
:109FA000FFF74AFC05EB44014870385D10F00F00E4
:109FB000FFF742FC05EB44018870002C01D0385DAE
:109FC0003618641C1A4F3878401CA042E4D2F6437D
:109FD00006F0FF0630000009FFF72EFC05EB4401F8
:109FE000487016F00F063000FFF726FC05EB440121
:109FF0008870032005EB4401C8706000001DF2BDAD
:10A00000011800F0021002000214020000A0054036
:10A0100000D000400080000C008000C0DC04002064
:10A02000D4040020800300200400FA050CED00E0B9
:10A0300000040020D80400208001002080020020BD
:10A0400038B50C000021C0B2FFF7D4FB05002D018C
:10A050002000C0B2FFF7CEFB45192800C0B232BDC8
:10A06000114340F8341F7047F8B504460E461746B2
:10A070001D4600F035F8B6EB071F04F1300005D29D
:10A08000016841F0200101607F0803E0026822F0CE
:10A0900020020260F600B6FBF7F0401C400804F115
:10A0A00024028109116000F03F0004F128010860DA
:10A0B00004F12C0004F1180105600020086020461E
:10A0C000BDE8F240FFE700F12C010A6842F01002FF
:10A0D0000A6040F2013150F8303F0B430360704793
:10A0E00000F118010A681307FCD400F12C010A687A
:10A0F00022F010020A6050F8303F02490B40036022
:10A1000070470000FEFCFFFF11430160704750F8EC
:10A11000302F22F01002F7E7002914BF40303C3006
:10A120000068704740F8441F704750F8482FEBE72D
:10A1300080B500202649086010212648FEF709FE58
:10A1400002212548FEF70FFE002024490860402127
:10A150002348FEF708FE002022490860FEF760FF52
:10A160002149086001202149086001BD10B51F4840
:10A17000006800282AD0FEF753FF1B490968401ADF
:10A180000A2823D300211A480068002801D051F082
:10A1900001010F4C0422174800F032F820602078AB
:10A1A000C00703D5144815490860FBE740200D4956
:10A1B00008604FF6FF70FFF7F2FC002803D0022082
:10A1C0000649086002E000200449086010BD000054
:10A1D000E404002000800540005002400850024086
:10A1E00000A0054000A10540E8040020E004002094
:10A1F00040800540C00400200400FA050CED00E09A
:10A2000070B40B00002503E050F8254023436D1C7B
:10A21000541EA542F8D300EB820454F8044C2340AA
:10A220000D00002603E050F826402540761C541E01
:10A23000A642F8D32B4300EB820444F8043C921E60
:10A2400006E000EB820454F8044C40F82240521E11
:10A25000002AF6D10160180070BC704710B507499C
:10A2600079441831064C7C44163404E00A68081D11
:10A27000114488470146A142F8D110BD2C000000CE
:10A28000380000004EF68851CEF20001086840F414
:10A2900070000860BFF34F8FBFF36F8F4FF00070F7
:10A2A000E1EE100A70470000ABF5FFFF3805000033
:10A2B000000000200000000080B5FEF7B4FEFFF7AC
:10A2C00037FFFDF7D3FFFFF7A3FCFEF756FFFFF7BD
:10A2D0004DFFFFF7FDFCF8E780B50448016851F435
:10A2E0007001016000F008F801BD000088ED00E099
:10A2F000FEE7FEE700BFFDE7AFF30080FFF7C2FF18
:10A3000000F000F800F00DF8002801D0FFF7A6FFDC
:10A31000AFF300800020AFF30080FFF7CDFF00F027
:10A3200002F80120704700F001B8000007463846E7
:10A3300000F002F8FBE7000080B5AFF30080024AAE
:10A3400011001820ABBEFBE726000200303132338B
:0CA3500034353637383941424344454625
:040000050000A2F95C
:00000001FF
